:0400000057EF00F0C6
:100008002B002B002B002B002B002B002B002B0090
:10001800D34B2B002B002B002B002B002B002B008D
:100028002B002B002B002B002B002B002B002B0070
:100038002B002B002B0015482B002B002B002B002E
:10004800104B2B002B002B002B002B002B002B0020
:100058002B002B002B002B002B002B002B002B0040
:100068002B002B002B002B002B002B002B002B0030
:10007800434B2B002B002B002B002B002B002B00BD
:100088002B002B002B002B002B002B002B002B0010
:100098002B002B002B002B002B002B002B002B0000
:0A00A8002B002B00FF0062EF93F025
:10F4F4000001000A006400E8031027010010000066
:10F5040001001020546573742033412065637269CF
:10F514007475726520426C6F6320313238204279F1
:10F52400746573206461746120656E20466C617338
:10F534006820617420402030783744303020736F65
:10F544006974203332303030200D0A002054657342
:10F554007437203A20656372697475726520426C51
:10F564006F632036342020574F5244206461746105
:10F5740020656E20466C61736820617420402030E1
:10F58400783744303020736F697420333230303030
:10F59400200D0A002055415254312048617264778D
:10F5A400617265205243363D545820205243373D02
:10F5B400525820203131353230302C382C4E2C31F9
:10F5C4002020496E7465727275707420486967688A
:10F5D40020737572205258200D0A002054657374EC
:10F5E4003220656372697475726520426C6F6320A2
:10F5F4003634204279746573206461746120656EC9
:10F6040020466C6173682061742040203078374450
:10F61400303020736F6974203332303030200D0A5B
:10F62400002054657374203141203A204566666198
:10F63400636520426C6F63203132382042797465EF
:10F64400732020656E20466C6173682061742040CD
:10F654002030783744303020736F6974203332306F
:10F664003030200D0A000D0A2E2E5361697369652E
:10F6740020657420656E766F6920666963686965C4
:10F6840072202A2E77617620766961205445524192
:10F694005445524D207465726D696E616C205365DA
:10F6A4006E642066696C650D0A00205465737435B8
:10F6B400203A2045666661636520426C6F632031A1
:10F6C40032382042797465732020656E20466C615F
:10F6D40073682061742040203078374430302073C0
:10F6E4006F6974203332303030200D0A00205465A5
:10F6F40073742034412052652D4C656374757265B2
:10F704002031323820427974657320656E2020469A
:10F714006C61736820617420402030783744303045
:10F7240020736F6974203332303030200D0A002D7D
:10F734002D2D2D2D2D2066696E2064752031657266
:10F74400205465737420466C617368202E2E2061EA
:10F75400647265737361676520466C617368206DBC
:10F764006F64756C6F20776F7264202D2D2D720A73
:10F77400002D2D2D2066696E2064752032656D2064
:10F784005465737420466C617368202E2E20616466
:10F794007265737361676520466C617368206D6F71
:10F7A40064756C6F20427974652D2D2D2D2D2D0DD2
:10F7B4000A00205465737438203A2052652D4C6534
:10F7C400637475726520363420574F524420656E39
:10F7D4002020466C617368206174204020307837A3
:10F7E40044303020736F6974203332303030200D50
:10F7F4000A002072652053746172742043435031AF
:10F804002050574D3120386269747320617420315F
:10F8140031303235206F6E205243312C20647574A0
:10F82400793D6B3D76616C756520353132200D0A6A
:10F83400002D2D2D2D2032656D20205465737420EC
:10F84400466C617368202E2E206164726573736147
:10F85400676520466C617368206D6F64756C6F20FA
:10F8640042797465202D2D2D2D2D2D2D0D0A00206E
:10F8740054657374332052652D4C656374757265D9
:10F8840020427974657320656E2020466C6173682C
:10F8940020617420402030783744303020736F6901
:10F8A40074203332303030200D0A002044757479CE
:10F8B4002076616C756520617520636C617669657D
:10F8C4007220206B3D58585858202831303234204B
:10F8D400706F757220736F7274697220647520740E
:10F8E400657374200D0A002054657374203241201E
:10F8F4004C656374757265203132382042797465C1
:10F904007320466C6173682061742040203078371E
:10F9140044303020736F6974203332303030200D1E
:10F924000A0020496E697420436F6D7074657572A6
:10F93400203234206269747320534D54312C206278
:10F944006173652064652074656D7073203A204688
:10F954004F53432036344D487A0D0A0020546573C2
:10F964007436203A204C65637475726520363420F1
:10F97400576F726420466C61736820617420402064
:10F9840030783744303020736F697420333230302C
:10F9940030200D0A00205465737431204C65637463
:10F9A40075726520363420427974657320466C6123
:10F9B40073682061742040203078374430302073DD
:10F9C4006F6974203332303030200D0A00205072B9
:10F9D4006F6A6574204D504C414258203A31384684
:10F9E40032374B34325F546573745F4563725F4CD6
:10F9F40065635F466C6173685F323032322D303933
:10FA04002E580D0A000D0A2E2E2E2E76657269666A
:10FA140020467265712E2050574D203D3930B55324
:10FA2400202C2070656E64616E74202074696D658D
:10FA34006F75742032307365630D0A00205573614D
:10FA440067652064652054696D6572322065742091
:10FA54004343503120706F75722050574D2031311F
:10FA640030323520487A20737572205243310D0AA2
:10FA74000020436F6D70696C65206C6520257320D0
:10FA840061202573205554430D0A20617665632057
:10FA940076657273696F6E20584338203A202025AA
:10FAA400640D0A00204861726477617265203A200F
:10FAB40050494331384632374B3432202C20464F9C
:10FAC400534320696E7465726E65203D36344D482B
:10FAD4007A200D0A0020546573742054696D657290
:10FAE4003420206465636F6D7074652073757220B3
:10FAF400343020626F75636C657320287831303040
:10FB04006D53290D0A0020557361676520646520D3
:10FB140054696D657231207820666F6973203130C5
:10FB2400306D53202C2054696D657234202031309F
:10FB3400306D530D0A00204166666963686167652C
:10FB440020446174617320626C6F6373202873694D
:10FB5400205242313D3029202076616C6575722037
:10FB64005242313D2000202020204A6F7565206CD0
:10FB740065206669636869657220776176652031FE
:10FB84003130323520487A20656E2038206269741D
:10FB940073200D0A002044757265652072656C65DA
:10FBA400637475726520313238206279746573200C
:10FBB400656E20666C61736820203A005465737426
:10FBC4002054696D6572312061726D6520706F75A6
:10FBD400722033302078203130306D7365630D0A24
:10FBE4000020457461706520300D0A2E2E2041746A
:10FBF40074656E7465202049542052582055415232
:10FC040054310D0A002053746F7020534D54312029
:10FC140020204E62205469637320617665632075E9
:10FC24006C746F61202D3E20000D0A202D2D2D2D8A
:10FC34002D2D2D2066696E206465207465737473A0
:10FC4400202D2D2D2D2D2D200D0A000D0A202D2DBA
:10FC54002D2D2D2D2D2D2D2D2D2D2D2D2D2D2D2DD0
:10FC64002D2D2D2D2D2D2D2D2D0D0A002041726DA4
:10FC7400652049565420696E746572727570747388
:10FC8400202031384632374B34320D0A00206C655F
:10FC94006374757265206465732064617461732094
:10FCA4003A202535642062797465730D0A0020209A
:10FCB400476C6F62616C2046696C652073697A6574
:10FCC400203D202535642062797465730D0A000D8A
:10FCD4000A4365206E276573742070617320756E06
:10FCE40020574156202121212E2E2E0D0A00204579
:10FCF400746170652033203B206C65637475726594
:10FD040020646573206461746173203A000D0A20D5
:10FD140046696E206465206C656374757265206441
:10FD240061746120776176650D0A00205461696C05
:10FD34006C652044617461203D202535642062791E
:10FD4400746573200D0A00206E65772050574D208E
:10FD540064757479206379636C65203D202535646E
:10FD64000D0A0020467265712E20456368616E7429
:10FD7400696C6C2E3D2025356420487A0D0A000DEF
:10FD84000A205265E775202535642062797465730D
:10FD9400200D0A202573200D0A004574617065202A
:10FDA40032202020466F726D6174206368756E6B1B
:10FDB400203A0D0A000D0A20426C6F63202325357A
:10FDC4006420204F66667365743D2535640D0A0012
:10FDD400205461696C6C6520426C6F63203D202562
:10FDE40035642042797465730D0A0020496E697484
:10FDF4002043435020504D5731206F6E20524331E1
:10FE04000D0A002046696368696572205741566689
:10FE14006D7420202E2E4F4B0D0A000D0A207265A2
:10FE240073746520647520426C6F63202331200D48
:10FE34000A002056657273696F6E203A20323032A0
:10FE4400322D303931320D0A000D0A20496E6974A1
:10FE54002054696D65723220203930B5530D0A0083
:10FE6400205465737420534D5431207375722031BE
:10FE7400306D53203A20002054696D657231206939
:10FE84006E6974203130306D53200D0A000D0A2044
:10FE94002D2D2D2D2D454E44202D2D2D2D2D200D78
:10FEA4000A0020476C6F62616C2046696C652073A0
:10FEB400697A65203D200020466F726D6174205080
:10FEC400434D203D202535640D0A00204E62204319
:10FED400616E6175784D203D202535640D0A002042
:10FEE4004D617820426C6F6373203D253564200D8D
:10FEF4000A00457461706520320D0A205265E77569
:10FF0400203A0D0A002046696368696572205249E7
:10FF1400464620210D0A0030313233343536373825
:10FF24003961626364656600207265746F7572205E
:10FF34006B3D2535640D0A00205461696C6C6520A5
:10FF440044617461203D2000205461696C6C65201B
:10FF5400426C6F63203D0020426C6F632023253583
:10FF640064200D0A002045746170652035200D0A57
:10FF7400005365702031322032303232000D0A20B5
:10FF840053746F700D0A002041726D65200D0A00D4
:10FF94000D0A53746F700D0A002053746172740D4E
:10FFA4000A00206A3D202535642000202C20736F30
:10FFB4006974200057415645666D74200031373A04
:10FFC40033303A323900202575202D3E2000307818
:10FFD400253032782E003078253034782E00286E83
:10FFE400756C6C290020253032782E002075530D55
:0BFFF4000A005249464600203E000073
:020000040001F9
:10000000600E3901D96F000EDB6F000EDD6F080E38
:10001000DF6F000EDE6F290E0001C06F960EBF6FFE
:100020007F0EE82EFED7BF2FFCD7C02FFAD7900E39
:100030003C01E56F030EE66F290E0001C06F960EBE
:10004000BF6F7F0EE82EFED7BF2FFCD7C02FFAD789
:1000500000EC95F0000E3E01BC6F000EBD6F81EC10
:1000600097F0000E566E7F0E556E000E586E000E05
:10007000576E45EF80F0000E5724D96E010E5820C0
:10008000DA6E000EDF6E574A582A5550575C5650AC
:100090005858D8A04EEF80F050EF80F03BEF80F042
:1000A000000E586E000E576E800E5724D96E010E4A
:1000B0005820DA6E000EDF6E574A582A585009E170
:1000C0004F0E575CD8A067EF80F069EF80F054EFD7
:1000D00080F0000E586E000E576E000E5724D96E39
:1000E000020E5820DA6E000EDF6E574A582A58501A
:1000F00009E17F0E575CD8A080EF80F082EF80F09E
:100100006DEF80F0000E4F6E020E506E36EC97F0E1
:10011000000E4F6E020E506E60003FF1D9FF60007E
:1001200043F1DAFF000EDF6E7AEC98F0000E00016A
:10013000976F000E966F000E936F000E926F000E79
:10014000916F0A0E906F000E8D6F000E8C6F000E77
:10015000B56F7AEC98F0D10E026EF90E036EE1ECF9
:1001600096F0360E026EFE0E036EE1EC96F04FC076
:100170000EF050C00FF0750E106EFA0E116E750E67
:10018000126EFF0E136EC10E146EFF0E156E090E69
:10019000176E380E166ED3EC8BF00EC055F00FC0F4
:1001A00056F04FC026F050C027F0B3EC95F0A80EE3
:1001B000026EFA0E036EE1EC96F0980E026EF50EEA
:1001C000036EE1EC96F00A0E026EFB0E036EE1EC9C
:1001D00096F0400E026EFA0E036EE1EC96F07AECA9
:1001E00098F0010E0001B26F260E026EF90E036E3A
:1001F000E1EC96F046EC98F0000E0001BB6F000EAB
:10020000BC6F000EBD6F000EBE6FBB0E476E000EC2
:10021000486E3F01219521932191640E026EFE0EDE
:10022000036EE1EC96F03F01208B1F8FD00E000192
:10023000BF6FC90EE82EFED7BF2FFCD700D03F01FD
:100240001F9F60001FF1D9FF600023F1DAFF6F00EC
:100250004BFCDFFF20EE01F04750D9264850DA2250
:100260006F004FFCDFFF20EE02F04750D9264850C8
:10027000DA226F0053FCDFFF20EE03F04750D9264F
:100280004850DA22000EDF6E090E026EFC0E036E7D
:10029000E1EC96F04FC00FF050C010F0BBC011F071
:1002A000BCC012F0BDC013F0BEC014F0000E166E3C
:1002B0000A0E156E69EC91F04FC026F050C027F081
:1002C000B3EC95F0AF0E026EFF0E036EE1EC96F00C
:1002D0003F0121A56EEF81F070EF81F07CEF81F09E
:1002E000D8900001BB35686FBC35696FBD356A6F4A
:1002F000BE356B6F98EF81F0BBC0BFF0BCC0C0F0E3
:10030000BDC0C1F0BEC0C2F0050E8DEF81F000018E
:10031000D890C233C133C033BF33E82E87EF81F0AA
:10032000BFC068F0C0C069F0C1C06AF0C2C06BF065
:10033000800E1C6E010E1D6E68C01EF069C01FF09D
:100340006AC020F06BC021F0000E236E0A0E226EF0
:10035000EBEC95F01CC026F01DC027F0B3EC95F037
:10036000F00E026EFF0E036EE1EC96F07AEC98F060
:100370007AEC98F0990E026EF90E036EE1EC96F0AD
:10038000000E586E000E576E0F0E57140001BF6F0F
:10039000000E5814C06FBF51C011D8A4D2EF81F025
:1003A000D4EF81F0F4EF81F07AEC98F0800E0E6ECD
:1003B000010E0F6ECA0E106EFF0E116E57C0BFF009
:1003C00058C0C0F0D8900001BF37C037000EBF251D
:1003D000126E7D0EC021136ED3EC8BF0800E266E54
:1003E000010E276EB3EC95F0000E0001BF6F7D0E7D
:1003F000C06F57C0C1F058C0C2F0D890C137C237E3
:10040000BF51C127C051C223C1C002F0C2C003F016
:10041000046A056ABBEC98F05B6E800E0E6E010EEE
:100420000F6ED20E106EFF0E116E5BC012F0136ACB
:10043000D3EC8BF0800E266E010E276EB3EC95F098
:10044000574A582A585009E1400E575CD8A02BEF64
:1004500082F02DEF82F0C4EF81F07AEC98F07AEC24
:1004600098F0DF0E026EF50E036EE1EC96F0000ED2
:10047000076E7D0E086E000E096E000E0A6E800E6D
:100480000B6E020E0C6EF8EC91F0556E566A55BE6E
:1004900056064FC00EF050C00FF02C0E106EFF0E1F
:1004A000116E55C012F056C013F0D3EC8BF04FC054
:1004B00026F050C027F0B3EC95F07AEC98F0730E6C
:1004C000026EF80E036EE1EC96F0000E586E000E10
:1004D000576E0F0E57140001BF6F000E5814C06FF7
:1004E000BF51C011D8A477EF82F079EF82F099EF75
:1004F00082F07AEC98F0800E0E6E010E0F6ECA0E2E
:10050000106EFF0E116E57C0BFF058C0C0F0D890EB
:100510000001BF37C037000EBF25126E7D0EC0210F
:10052000136ED3EC8BF0800E266E010E276EB3ECAB
:1005300095F0000E0001BF6F7D0EC06F57C0C1F077
:1005400058C0C2F0BF51C127C051C223C1C002F080
:10055000C2C003F0046A056ABBEC98F05B6E800EC3
:100560000E6E010E0F6ED20E106EFF0E116E5BC07E
:1005700012F0136AD3EC8BF0800E266E010E276EFC
:10058000B3EC95F0574A582A585009E1400E575C91
:10059000D8A0CDEF82F0CFEF82F069EF82F07AEC55
:1005A00098F07AEC98F0AE0E026EF60E036EE1EC67
:1005B00096F0000E026E7D0E036E000E046E000EAD
:1005C000056ECAEC97F07AEC98F0600E026EF90EA8
:1005D000036EE1EC96F0000E586E000E576E0F0E93
:1005E00057140001BF6F000E5814C06FBF51C011E7
:1005F000D8A4FDEF82F0FFEF82F01FEF83F07AECDA
:1006000098F0800E0E6E010E0F6ECA0E106EFF0E69
:10061000116E57C0BFF058C0C0F0D8900001BF376E
:10062000C037000EBF25126E7D0EC021136ED3ECB5
:100630008BF0800E266E010E276EB3EC95F0000E47
:100640000001BF6F7D0EC06F57C0C1F058C0C2F02F
:10065000D890C137C237BF51C127C051C223C1C0D2
:1006600006F0C2C007F0086A096AECEC97F006C011
:1006700055F007C056F0800E0E6E010E0F6EDA0EAA
:10068000106EFF0E116E55C012F056C013F0D3EC71
:100690008BF0800E266E010E276EB3EC95F0574A54
:1006A000582A585009E1400E575CD8A05AEF83F001
:1006B0005CEF83F0EFEF82F07AEC98F07AEC98F050
:1006C000500E026EF50E036EE1EC96F0000E076E12
:1006D0007D0E086E000E096E000E0A6E000E0B6E87
:1006E000030E0C6EF8EC91F0556E566A55BE560628
:1006F0004FC00EF050C00FF02C0E106EFF0E116E9A
:1007000055C012F056C013F0D3EC8BF04FC026F05A
:1007100050C027F0B3EC95F07AEC98F0B60E026E6C
:10072000F70E036EE1EC96F0000E586E000E576E59
:100730000F0E57140001BF6F000E5814C06FBF5149
:10074000C011D8A4A6EF83F0A8EF83F0C8EF83F020
:100750007AEC98F0800E0E6E010E0F6ECA0E106EBF
:10076000FF0E116E57C0BFF058C0C0F0D890000106
:10077000BF37C037000EBF25126E7D0EC021136E2D
:10078000D3EC8BF0800E266E010E276EB3EC95F045
:10079000000E0001BF6F7D0EC06F57C0C1F058C082
:1007A000C2F0D890C137C237BF51C127C051C22350
:1007B000C1C006F0C2C007F0086A096AECEC97F005
:1007C00006C055F007C056F0800E0E6E010E0F6E7B
:1007D000DA0E106EFF0E116E55C012F056C013F0F7
:1007E000D3EC8BF0800E266E010E276EB3EC95F0E5
:1007F000574A582A585009E1400E575CD8A003EFD9
:1008000084F005EF84F098EF83F07AEC98F0330EE3
:10081000026EF70E036EE1EC96F07AEC98F07AEC4B
:1008200098F0350E026EF80E036EE1EC96F07AEC5D
:1008300098F0250E026EF60E036EE1EC96F0000EB7
:10084000026E7D0E036E000E046E000E056ECAEC85
:1008500097F07AEC98F07AEC98F0EB0E026EF80EC6
:10086000036EE1EC96F0000E586E000E576E0F0E00
:1008700057140001BF6F000E5814C06FBF51C01154
:10088000D8A445EF84F047EF84F05FEF84F07AEC72
:1008900098F0800E0E6E010E0F6ECA0E106EFF0ED7
:1008A000116E000E5724126E7D0E5820136ED3EC7D
:1008B0008BF0800E266E010E276EB3EC95F0000EC5
:1008C0000001BF6F7D0EC06F57C0C1F058C0C2F0AD
:1008D000BF51C127C051C223C1C002F0C2C003F042
:1008E000046A056ABBEC98F05B6E800E0E6E010E1A
:1008F0000F6ED20E106EFF0E116E5BC012F0136AF7
:10090000D3EC8BF0800E266E010E276EB3EC95F0C3
:10091000574A582A585009E1800E575CD8A093EFE7
:1009200084F095EF84F037EF84F07AEC98F07AEC6D
:1009300098F0070E026EF50E036EE1EC96F0000ED5
:10094000076E7D0E086E000E096E000E0A6E800E98
:100950000B6E020E0C6EF8EC91F0556E566A55BE99
:1009600056064FC00EF050C00FF02C0E106EFF0E4A
:10097000116E55C012F056C013F0D3EC8BF04FC07F
:1009800026F050C027F0B3EC95F07AEC98F07AECB2
:1009900098F0F10E026EF60E036EE1EC96F0000E8A
:1009A0000001BB6F000EBC6F000EBD6F000EBE6F6E
:1009B0003F01208B1F8F000E586E000E576E000EE9
:1009C0000001BF6F7D0EC06F57C0C1F058C0C2F0AC
:1009D000BF51C127C051C223C1C002F0C2C003F041
:1009E000046A056ABBEC98F05B6E574A582A585067
:1009F00009E1800E575CD8A000EF85F002EF85F08A
:100A0000DFEF84F03F011F9F60001FF1D9FF6000FE
:100A100023F1DAFF6F004BFCDFFF20EE01F04750BF
:100A2000D9264850DA226F004FFCDFFF20EE02F09B
:100A30004750D9264850DA226F0053FCDFFF20EEE2
:100A400003F04750D9264850DA22000EDF6E7AECC8
:100A500098F0990E026EFB0E036EE1EC96F0BBC0AF
:100A6000BFF0BCC0C0F0BDC0C1F0BEC0C2F0050E3A
:100A700040EF85F00001D890C233C133C033BF339B
:100A8000E82E3AEF85F0BFC068F0C0C069F0C1C081
:100A90006AF0C2C06BF0800E1C6E010E1D6E68C045
:100AA0001EF069C01FF06AC020F06BC021F0000E7C
:100AB000236E0A0E226EEBEC95F01CC026F01DC0D2
:100AC00027F0B3EC95F0F00E026EFF0E036EE1EC32
:100AD00096F07AEC98F07AEC98F0750E026EF70EBC
:100AE000036EE1EC96F07AEC98F07AEC98F0000E58
:100AF0000001976F000E966F000E4F6E020E506E43
:100B000060003FF1D9FF600043F1DAFF000EDF6EB5
:100B10007AEC98F081EC97F0B290A09E3901A19107
:100B2000700E026EFC0E036EE1EC96F039019387B5
:100B3000949197819191D28CD28E7B0E026EFE0E93
:100B4000036EE1EC96F05CEC97F0C00E026EFB0ECB
:100B5000036EE1EC96F0000E036E1E0E026ECCECFE
:100B600098F08B0E026EFF0E036EE1EC96F0000122
:100B700094519511D8B4BFEF85F0C1EF85F0B7EF70
:100B800085F08AC055F08BC056F055C009F056C0AC
:100B90000AF0000E0C6E0A0E0B6E54EC96F0095023
:100BA000300F5B6E5B50E9EC98F0000E0001956F22
:100BB000000E946F59A2DFEF85F0E1EF85F0B7EFFB
:100BC00085F05992B290810E026EFF0E036EE1EC39
:100BD00096F07AEC98F0D90E026EFA0E036EE1EC04
:100BE00096F09D0E026EFF0E036EE1EC96F0000E85
:100BF0000001936F000E926F000E8F6F000E8E6FCC
:100C0000000E916F280E906F0BEC98F000018E5142
:100C10008F11D8B40EEF86F010EF86F006EF86F055
:100C200090C055F091C056F055C009F056C00AF07A
:100C3000000E0C6E0A0E0B6E54EC96F00950300F3D
:100C40005B6E5B50E9EC98F0000E00018F6F000EB8
:100C50008E6F59A82EEF86F030EF86F006EF86F003
:100C6000940E026EFF0E036EE1EC96F07AEC98F0B3
:100C70007AEC98F0EF0E026EFD0E036EE1EC96F04A
:100C8000DBEC98F04D0E026EFE0E036EE1EC96F07A
:100C900091EC98F0000E566E800E556E800E7C6EB4
:100CA000000E7D6E7AEC98F0090E026EFA0E036E5D
:100CB000E1EC96F0AF0E026EF80E036EE1EC96F0EA
:100CC000000E546E000E536E000E5A6E5CEC97F0E0
:100CD0003CEC94F0000E036EC80E026ECCEC98F063
:100CE000525007E1060E515CD8B079EF86F07BEFE9
:100CF00086F082EF86F059A280EF86F082EF86F0D0
:100D000070EF86F059B287EF86F089EF86F0EEEF4C
:100D100086F04FC00EF050C00FF0830E106EFD0E27
:100D2000116E51C012F052C013F0000E146E010E7D
:100D3000156ED3EC8BF04FC026F050C027F0B3EC0B
:100D400095F06B0E01010019D8A4A9EF86F0ABEF66
:100D500086F0EEEF86F03D0E0119D8A4B2EF86F0D2
:100D6000B4EF86F0EEEF86F0000E026E010E036E19
:100D700029EC98F0035009E1060E025CD8A0C3EFFD
:100D800086F0C5EF86F0EEEF86F0BA86000E010120
:100D9000066F020E086E010E096ED1EC90F008C0CD
:100DA00055F009C056F0600057F17CFF5650030B18
:100DB0007D6E4FC00EF050C00FF04B0E106EFD0E4A
:100DC000116E55C012F056C013F0D3EC8BF04FC02B
:100DD00026F050C027F0B3EC95F0BA96040E565C9E
:100DE000D8A0F5EF86F0F7EF86F066EF86F0BC8AC4
:100DF0006A0E026EF60E036EE1EC96F0000E546E73
:100E0000000E536E000E5A6EC1EF8BF0BC8AA6EF37
:100E10008BF07AEC98F0E50E026EFB0E036EE1ECBF
:100E200096F0000E526E000E516E3CEC94F0520E95
:100E30000001C06F2B0EBF6F000EE82EFED7BF2F34
:100E4000FCD7C02FFAD700F0C1EF8BF0F60E026E80
:100E5000FE0E036EE1EC96F0800E026E010E036E44
:100E6000000E046E010E056E000E076E400E066E3B
:100E7000AFEC93F0800E266E010E276EB3EC95F06A
:100E80007AEC98F0000E2C6E010E2D6E000E2F6E77
:100E9000400E2E6E27EC8FF0800E026E010E036E58
:100EA000F60E046EFF0E056E7AEC95F0000E0E6ED7
:100EB000010E0F6E800E106E010E116E65EC92F039
:100EC0000EC04DF00FC04EF04D504E10D8B46BEF29
:100ED00087F06DEF87F002EF87F0090E026EFF0ECC
:100EE000036EE1EC96F0A60E026EFE0E036EE1ECD0
:100EF00096F020EE05F04D50D9264E50DA22DF5004
:100F00000001BF6FBF51556E566A5550566E556AF7
:100F100020EE04F04D50D9264E50DA22DF50BF6F3C
:100F2000BF515524C06F000E5620C16F080EC0255A
:100F3000556E000EC121566E55C049F056C04AF09C
:100F4000800E0E6E010E0F6EB20E106EFC0E116E44
:100F500049C012F04AC013F0D3EC8BF0800E266E1D
:100F6000010E276EB3EC95F0800E026E010E036E3B
:100F7000B80E046EFF0E056E7AEC95F0080E0E6E3C
:100F8000010E0F6E800E106E010E116E65EC92F068
:100F90000EC04DF00FC04EF04D504E10D8B4D3EFF0
:100FA00087F0D5EF87F0ECEF87F0070E026EFE0EAC
:100FB000036EE1EC96F0090E0001C06F1E0EBF6FCC
:100FC000E40EE82EFED7BF2FFCD7C02FFAD700F0D3
:100FD000030E5A6EC1EF8BF0800E0E6E010E0F6E77
:100FE000A60E106EFF0E116EAEC012F0AFC013F061
:100FF000D3EC8BF0800E266E010E276EB3EC95F0CD
:101000007AEC98F0000E5A6E000E546E000E536E7D
:10101000D30E026EFC0E036EE1EC96F0C1EF8BF086
:101020007AEC98F0000E4D6E010E4E6E9E0E026E22
:10103000FD0E036EE1EC96F04C0E026EFF0E036E99
:10104000E1EC96F0100E4D6E010E4E6E800E026EAB
:10105000010E036E4DC004F04EC005F0000E076E89
:10106000040E066EB4EC96F020EE01F04D50D92639
:101070004E50DA22DF500001BF6FBF51556E566AE5
:101080005550566E556A600037F1D9FF60003BF14C
:10109000DAFFDF50BF6FBF515524556E000E56204A
:1010A000566E800E0E6E010E0F6ED40E106EFD0E7B
:1010B000116E55C012F056C013F0D3EC8BF0800EB9
:1010C000266E010E276EB3EC95F07AEC98F0140EB4
:1010D0004D6E010E4E6E800E026E010E036E4DC0FF
:1010E00004F04EC005F0000E076E020E066EB4EC62
:1010F00096F04DC02CF04EC02DF0000E2F6E020E5B
:101100002E6E27EC8FF020EE01F04D50D9264E5078
:10111000DA22DF500001BF6FBF51556E566A55503D
:10112000566E556A600037F1D9FF60003BF1DAFF77
:10113000DF50BF6FBF515524556E000E5620566EBE
:10114000800E0E6E010E0F6EBB0E106EFE0E116E37
:1011500055C012F056C013F0D3EC8BF0800E266E03
:10116000010E276EB3EC95F07AEC98F0160E4D6EEA
:10117000010E4E6E800E026E010E036E4DC004F025
:101180004EC005F0000E076E020E066EB4EC96F02F
:101190004DC02CF04EC02DF0000E2F6E020E2E6EA4
:1011A00027EC8FF020EE01F04D50D9264E50DA2278
:1011B000DF500001BF6FBF51556E566A5550566ED5
:1011C000556A600037F1D9FF60003BF1DAFFDF506C
:1011D000BF6FBF515524556E000E5620566E800EBF
:1011E0000E6E010E0F6ECF0E106EFE0E116E55C0FC
:1011F00012F056C013F0D3EC8BF0800E266E010E69
:10120000276EB3EC95F0180E4D6E010E4E6E800EEB
:10121000026E010E036E4DC004F04EC005F0000ECC
:10122000076E040E066EB4EC96F04DC02CF04EC066
:101230002DF0000E2F6E040E2E6E27EC8FF020EE98
:1012400001F04D50D9264E50DA22DF500001BF6F19
:10125000BF51556E566A5550566E556A600037F14B
:10126000D9FF60003BF1DAFFDF50BF6FBF5155245B
:10127000556E000E5620566E800E0E6E010E0F6ECD
:10128000670E106EFD0E116E55C012F056C013F0B1
:10129000D3EC8BF0800E266E010E276EB3EC95F02A
:1012A000FB0E026EFF0E036EE1EC96F0240E4D6E07
:1012B000010E4E6E600037F1D9FF60003BF1DAFF9E
:1012C000DF50E9EC98F020EE01F04D50D9264E5059
:1012D000DA22DF50E9EC98F020EE02F04D50D926EA
:1012E0004E50DA22DF50E9EC98F020EE03F04D503A
:1012F000D9264E50DA22DF50E9EC98F0800E026ECB
:10130000010E036E4DC004F04EC005F0000E076ED6
:10131000040E066EB4EC96F07AEC98F04DC02CF00A
:101320004EC02DF0000E2F6E040E2E6E27EC8FF0A7
:101330007AEC98F03C0E026EFF0E036EE1EC96F034
:10134000280E4D6E010E4E6E800E026E010E036E63
:101350004DC004F04EC005F0000E076E040E066E80
:10136000B4EC96F0800E2C6E010E2D6E000E2F6EDA
:10137000040E2E6E27EC8FF020EE01F04D50D92692
:101380004E50DA22DF500001BF6FBF51556E566AD2
:101390005550566E556A600037F1D9FF60003BF139
:1013A000DAFFDF50BF6FBF515524556E000E562037
:1013B000566E55C049F056C04AF0800E0E6E010EB2
:1013C0000F6E2F0E106EFD0E116E55C012F056C02E
:1013D00013F0D3EC8BF0800E266E010E276EB3EC6B
:1013E00095F055C0BFF056C0C0F0060E0001C16FA9
:1013F000D890C033BF33C12FF8EF89F0BFC086F05B
:10140000C0C087F0800E0E6E010E0F6EE30E106EE0
:10141000FE0E116E55C012F056C013F0D3EC8BF0D7
:10142000800E266E010E276EB3EC95F07AEC98F0E4
:10143000040E5A6E000E546E000E536E000E526E65
:10144000000E516E000E566E000E556EC1EF8BF001
:10145000BC8AF20E026EFC0E036EE1EC96F0800E7A
:101460000E6E010E0F6E910E106EFC0E116E49C0C5
:1014700012F04AC013F0D3EC8BF0800E266E010EF2
:10148000276EB3EC95F07AEC98F0040E5A6E000ECD
:101490004C6E010E4B6E1F0E026EFE0E036EE1ECE3
:1014A00096F02C0E4D6E010E4E6E4DC02CF04EC0BF
:1014B0002DF0000E2F6E140E2E6E27EC8FF07AECAE
:1014C00098F03A0E026EFB0E036EE1EC96F0CBB292
:1014D0006CEF8AF06FEF8AF0010E70EF8AF0000E69
:1014E000300F5B6E5B50E9EC98F07AEC98F07AEC98
:1014F00098F0000E546E400E536E000E526E000EA9
:10150000516E520E0001C06F2B0EBF6F000EE82E01
:10151000FED7BF2FFCD7C02FFAD700F0F4EF8AF028
:101520003CEC94F0040E0001C06FA80EBF6F0B0ED0
:10153000E82EFED7BF2FFCD7C02FFAD700D000016E
:10154000B505D8A4A6EF8AF0A8EF8AF0F4EF8AF0E8
:101550004B4A4C2A000ECBB2010E5B6E5B50D8A4F6
:10156000B4EF8AF0B6EF8AF0E0EF8AF0800E0E6EEC
:10157000010E0F6EB90E106EFD0E116E4BC012F003
:101580004CC013F0C00E5324146EFF0E5420156E81
:10159000D3EC8BF0800E266E010E276EB3EC95F027
:1015A000000E4D6E010E4E6E4DC02CF04EC02DF053
:1015B000000E2F6E400E2E6E27EC8FF0F4EF8AF0A7
:1015C000800E0E6E010E0F6E5B0E106EFF0E116E12
:1015D0004BC012F04CC013F0D3EC8BF0800E266E93
:1015E000010E276EB3EC95F0C00E0001BF6FFF0E29
:1015F000C06F49C0C1F04AC0C2F0BF51C127C0513D
:10160000C223C151535CC2515458D8B00AEF8BF079
:101610000CEF8BF017EF8BF086514B5C87514C58D9
:10162000D8A015EF8BF017EF8BF090EF8AF0110E2A
:10163000026EFD0E036EE1EC96F0BC8A050E5A6E4A
:10164000A30E0001C06F570EBF6F020EE82EFED72B
:10165000BF2FFCD7C02FFAD700F0C1EF8BF0000EE0
:101660000001AF6F000EAE6F690E026EFF0E036ECB
:10167000E1EC96F0F60E026EF70E036EE1EC96F0DA
:101680007E8EAC8E4F0E026EFC0E036EE1EC96F079
:101690006A0E026EFB0E036EE1EC96F0520E026EC5
:1016A000FC0E036EE1EC96F0000E7D6E000E586E9F
:1016B000000E576EBA86000E7D6E800E5724D96ECE
:1016C000030E5820DA6EDF507C6EC90E00D000D0B9
:1016D000E82EFCD700F0BA96574A582A1B0E585CE1
:1016E000D8A075EF8BF077EF8BF05AEF8BF0000EF0
:1016F0007D6E800E7C6EA30E0001C06F570EBF6F13
:10170000020EE82EFED7BF2FFCD7C02FFAD700F06D
:101710000001AE4BAF2BAF5109E1050EAE5DD8A075
:1017200094EF8BF096EF8BF042EF8BF0060E5A6E33
:10173000C1EF8BF07E9EAC9E2D0E026EFC0E036EF2
:10174000E1EC96F0070E5A6EC1EF8BF05A50000A8A
:10175000D8B409EF87F0010AD8B426EF87F0020A5F
:10176000D8B410EF88F0070AD8B428EF8AF0010A3D
:10177000D8B42FEF8BF0030AD8B49AEF8BF0C1EFF7
:101780008BF0050E5A64C7EF8BF0C9EF8BF006EFB4
:1017900087F0910E026EFE0E036EE1EC96F0CFEF35
:1017A0008BF057EF00F0000E1E6E000E1D6E120E35
:1017B000226E000E236E04EF8FF0250E2B18D8B486
:1017C000E4EF8BF0E6EF8BF0F5EF8BF060003BF091
:1017D000D9FF60003FF0DAFF6000AFF0DFFF0E4A94
:1017E0000F2A1D4A1E2A04EF8FF0000E2A6E000EEB
:1017F000296E000E286E00EF8CF02884104A112A02
:10180000600043F0F6FF600047F0F7FF000EF86E4F
:101810000800F550300AD8B4FDEF8BF010EF8CF0D3
:10182000600043F0F6FF600047F0F7FF000EF86E2F
:101830000800F55061EC98F0D8A021EF8CF023EF70
:101840008CF016EF8DF0000E2A6E000E296E29C066
:1018500002F02AC003F0000E056E0A0E046EA6EC1C
:1018600098F002C029F003C02AF0D00E186EFF0EC7
:10187000196E600043F0F6FF600047F0F7FF000EBE
:10188000F86E0800F5501A6E1B6A18501A26195087
:101890001B221A5029261B502A22104A112A6000A6
:1018A00043F0F6FF600047F0F7FF000EF86E080007
:1018B000F55061EC98F0D8B060EF8CF062EF8CF0EE
:1018C00027EF8CF016EF8DF0288E3FEF8DF0600043
:1018D0008BF0D9FF60008FF0DAFF6F0078FF20F007
:1018E0006F0074FF21F0020E2226000E23222050EA
:1018F0002110D8A47EEF8CF080EF8CF084EF8CF078
:10190000E20E206EFF0E216E000E256E000E246E7C
:101910008CEF8CF0244A252A24502024186E255060
:101920002120196E600063F0F6FF600067F0F7FF9A
:10193000000EF86E1F0EF76403D00800F55007D0B4
:101940006F00DBFFE9FF6F00DFFFEAFFEF500009E8
:10195000D8A4ADEF8CF0AFEF8CF08AEF8CF029506B
:10196000245C2A502558D8B0B8EF8CF0BAEF8CF030
:10197000C0EF8CF02450295E25502A5AD2EF8CF00B
:10198000000E2A6E000E296ED2EF8CF060003BF044
:10199000D9FF60003FF0DAFF200EDF6E0E4A0F2AFB
:1019A0001D4A1E2A2906D8A02A06292806E12A2827
:1019B000D8A4DDEF8CF0DFEF8CF0C6EF8CF003EFF6
:1019C0008DF0600083F0F6FF600087F0F7FF000EF7
:1019D000F86E60003BF0D9FF60003FF0DAFF1F0EA9
:1019E000F76403D00800F55007D06F00DBFFE9FF74
:1019F0006F00DFFFEAFFEF50DF6E204A212A0E4A18
:101A00000F2A1D4A1E2A2406D8A02506242806E1EE
:101A10002528D8A40EEF8DF010EF8DF0E1EF8CF0BB
:101A200004EF8FF0C00E28123FEF8DF0600043F0FE
:101A3000F6FF600047F0F7FF104A112A000EF86E1B
:101A400008006F00D4FF2BF02B50000AD8B41AEF17
:101A50008FF0640AD8B43FEF8DF00D0AD8B43FEF91
:101A60008DF01A0AD8B467EF8CF0060AD8B412EFDA
:101A70008DF00D0AD8B464EF8CF004EF8FF028C01D
:101A800018F0C00E1816D8A448EF8DF04AEF8DF06C
:101A900069EF8DF060008BF0D9FF60008FF0DAFF06
:101AA0006F0078FF26F06F0074FF27F0020E2226E9
:101AB000000E232227BE61EF8DF05FEF8DF0CBEF9C
:101AC0008DF0030E2812266C271ED8B0272ACBEFE4
:101AD0008DF060008BF0D9FF60008FF0DAFF6F00AF
:101AE00078FF26F06F0074FF27F0020E2226000E0A
:101AF0002322CBEF8DF0010E2B6E2B50020DF50E35
:101B0000F324F66EF40EF420F76EF86A000EF82255
:101B10000900F550265C0900F5502758D8B093EF1E
:101B20008DF095EF8DF097EF8DF0DBEF8DF02B2A98
:101B3000050E2B18D8A49FEF8DF0A1EF8DF07DEF4F
:101B40008DF0DBEF8DF0010E2B6E2B50020DFF0E92
:101B5000F324F66EF40EF420F76EF86A000EF82205
:101B60000900F550265C0900F5502758D8B0BBEFA6
:101B70008DF0BDEF8DF0BFEF8DF0DBEF8DF02B2AF8
:101B8000040E2B18D8A4C7EF8DF0C9EF8DF0A5EF88
:101B90008DF0DBEF8DF02850C00B000AD8B47BEF3E
:101BA0008DF0800AD8B4A3EF8DF0400AD8B47BEF53
:101BB0008DF0DBEF8DF029502A10D8B4E2EF8DF0D4
:101BC000E4EF8DF0F2EF8DF028C018F0030E181638
:101BD000D8B4EDEF8DF0EFEF8DF0F2EF8DF0290638
:101BE000D8A02A062B50186E196A2950185C195073
:101BF000800A1A6E2A50800A1A58D8B002EF8EF066
:101C000004EF8EF00AEF8EF02B50295E000E2A5A58
:101C10000EEF8EF0000E2A6E000E296E28A413EF30
:101C20008EF015EF8EF04FEF8EF028C018F0030EF7
:101C30001816D8B41EEF8EF020EF8EF02CEF8EF039
:101C400060003BF0D9FF60003FF0DAFF2D0EDF6E41
:101C50000E4A0F2A1D4A1E2A29502A10D8B433EFE3
:101C60008EF035EF8EF087EF8EF060003BF0D9FFFD
:101C700060003FF0DAFF300EDF6E0E4A0F2A1D4A79
:101C80001E2A2906D8A02A0629502A10D8A44BEFCC
:101C90008EF04DEF8EF035EF8EF087EF8EF02950FD
:101CA0002A10D8B456EF8EF058EF8EF070EF8EF009
:101CB00060003BF0D9FF60003FF0DAFF200EDF6EDE
:101CC0000E4A0F2A1D4A1E2A2906D8A02A06295084
:101CD0002A10D8A46EEF8EF070EF8EF058EF8EF0D1
:101CE00028C018F0030E1816D8B479EF8EF07BEFE9
:101CF0008EF087EF8EF060003BF0D9FF60003FF080
:101D0000DAFF2D0EDF6E0E4A0F2A1D4A1E2A2BC047
:101D10001FF0FBEF8EF01F50020DF50EF324F66E50
:101D2000F40EF420F76EF86A000EF82209006F0036
:101D3000D4FF04F00A006F00D4FF05F026C002F0C3
:101D400027C003F040EC95F002C009F003C00AF090
:101D5000000E0C6E0A0E0B6E54EC96F00950300F0C
:101D60002B6EEEEF8EF026C002F027C003F01F505E
:101D7000020DFF0EF324F66EF40EF420F76EF86AEF
:101D8000000EF82209006F00D4FF04F00A006F0073
:101D9000D4FF05F040EC95F002500F0B1C6E1B0EAB
:101DA0001C24F66EF76AFF0EF722F86A000EF8227E
:101DB00008006F00D4FF2BF0EEEF8EF02850C00B20
:101DC000000AD8B48BEF8EF0800AD8B4B3EF8EF04F
:101DD000400AD8B48BEF8EF0EEEF8EF060003BF04F
:101DE000D9FF60003FF0DAFF6000AFF0DFFF0E4A7E
:101DF0000F2A1D4A1E2A1F061F28D8A402EF8FF0A3
:101E000004EF8FF0DEEF8EF0600043F0F6FF60002D
:101E100047F0F7FF104A112A000EF86E08006F0015
:101E2000D4FF2BF02B50D8A418EF8FF01AEF8FF0BF
:101E3000DDEF8BF060003BF0D9FF60003FF0DAFF90
:101E4000000EDF6E1DC00EF01EC00FF012002EC07F
:101E500030F02FC031F0040E326ED8903132303273
:101E6000322E2DEF8FF030C03BF031C03CF02F50C0
:101E700007E1100E2E5CD8B040EF8FF042EF8FF0EC
:101E800077EF8FF0200EE9EC98F0000E446E000E14
:101E9000436E68EF8FF0330E0E6E000E0F6EE90E7C
:101EA000106EFF0E116E43502C24D96E44502D201D
:101EB000DA6EDF50306E3050126E136AD3EC8BF056
:101EC000330E266E000E276EB3EC95F0434A442A7B
:101ED0002E50435C2F504458D8A071EF8FF073EF11
:101EE0008FF04BEF8FF07AEC98F027EF90F0000E28
:101EF000426E000E416EC3EF8FF0200EE9EC98F0B9
:101F0000000E446E000E436E41C030F042C031F00E
:101F1000303A313AF00E311630500F0B3112F00ECC
:101F20003016435030243F6E44503120406E330E03
:101F30000E6E000E0F6EE90E106EFF0E116E3F500A
:101F40002C24D96E40502D20DA6EDF50306E305088
:101F5000126E136AD3EC8BF0330E266E000E276ED2
:101F6000B3EC95F0434A442A445009E1100E435C17
:101F7000D8A0BDEF8FF0BFEF8FF084EF8FF07AEC39
:101F800098F0414A422A3B50415C3C504258D8A00C
:101F9000CCEF8FF0CEEF8FF07DEF8FF03BC030F0C5
:101FA0003CC031F0303A313AF00E311630500F0B60
:101FB0003112F00E301630C03FF031C040F03F50CB
:101FC0002E5C3D6E40502F583E6E3D503E10D8B4B2
:101FD000ECEF8FF0EEEF8FF027EF90F0200EE9ECB2
:101FE00098F0000E426E000E416E1AEF90F0330E24
:101FF0000E6E000E0F6EE90E106EFF0E116E3F504A
:102000002C24306E40502D20316E41503024D96E3A
:1020100042503120DA6EDF50326E3250126E136A47
:10202000D3EC8BF0330E266E000E276EB3EC95F0DA
:10203000414A422A3D50415C3E504258D8A023EFCD
:1020400090F025EF90F0F7EF8FF073EF8FF07AECD0
:1020500098F012003901A3A730EF90F032EF90F022
:10206000D0EF90F093A737EF90F039EF90F0D0EFEA
:1020700090F06F00A0F7BAF03D01F9AB42EF90F09D
:1020800044EF90F04BEF90F0F99B0001A44BA52B8F
:102090006F00A0F7BAF03D01F9A751EF90F053EFB0
:1020A00090F059EF90F00001A44BA52B6F00A0F722
:1020B000BAF0000E5124D96E010E5220DA6E600083
:1020C000EBF2DFFFC00E53240001846FFF0E54209B
:1020D000856F84518511D8B470EF90F072EF90F055
:1020E00084EF90F01B0E855DD8B079EF90F07BEF18
:1020F00090F084EF90F0800E8425D96E030E852138
:10210000DA6E6000EBF2DFFF534A542A514A522A3A
:10211000C1EF90F0525009E1400E515CD8A093EF0E
:1021200090F095EF90F0D0EF90F0BC8A3901939742
:10213000010E0001B56F000E526E000E516E010EC1
:102140005A6ED0EF90F0525007E1400E515CD8B07B
:10215000ACEF90F0AEEF90F0B9EF90F05350495CD7
:1021600054504A58D8B0B7EF90F0B9EF90F0D0EF94
:1021700090F0BC8A39019397010E0001B56FD0EF42
:1021800090F05A50000AD8B48AEF90F0030AD8B4FD
:10219000A3EF90F0070AD8B4A3EF90F0D0EF90F03F
:1021A0001100D5EF90F0084A092A600023F0D9FF0A
:1021B000600027F0DAFF200EDE18D8B4E2EF90F0CE
:1021C000E4EF90F0D3EF90F0600023F0D9FF6000CF
:1021D00027F0DAFF090EDE18D8B4F1EF90F0F3EF34
:1021E00090F0D3EF90F0000E0E6E000E0D6E000E0C
:1021F0000C6E600023F0D9FF600027F0DAFF2D0E8F
:10220000DE18D8A406EF91F008EF91F00DEF91F0F1
:102210000C2A084A092A3EEF91F0600023F0D9FF0A
:10222000600027F0DAFF2B0EDE18D8A41AEF91F029
:102230001CEF91F03EEF91F0084A092A3EEF91F031
:102240000DC002F00EC003F0000E056E0A0E046E03
:10225000A6EC98F0600023F0D9FF600027F0DAFFC9
:10226000DF500A6E0A500226000E0322D00E02240E
:102270000D6EFF0E03200E6E1CEF91F0600023F038
:10228000D9FF600027F0DAFFDF5061EC98F0D8B09A
:102290004CEF91F04EEF91F020EF91F00C50D8B44C
:1022A00054EF91F056EF91F064EF91F00DC00AF009
:1022B0000EC00BF00A1E0B1E0A4A0B2A0AC008F0B9
:1022C0000BC009F068EF91F00DC008F00EC009F0E6
:1022D000120011C017F012C018F013C019F014C08A
:1022E0001AF017C002F018C003F019C004F01AC0A9
:1022F00005F015C006F016C007F0000E07BEFF0E71
:10230000086E096E10EC93F002C017F003C018F0CD
:1023100004C019F005C01AF00F4A102A17501810FF
:1023200019101A10D8A497EF91F099EF91F071EF6E
:1023300091F060003FF0D9FF600043F0DAFF000E3B
:10234000DF6E0F06D8A0100611C002F012C003F015
:1023500013C004F014C005F015C006F016C007F055
:10236000000E07BEFF0E086E096EF8EC93F00250E7
:102370001B6E11C002F012C003F013C004F014C0B1
:1023800005F015C006F016C007F0000E07BEFF0EE0
:10239000086E096E10EC93F002C011F003C012F049
:1023A00004C013F005C014F0090E1B64DAEF91F0BD
:1023B000DCEF91F0DEEF91F0070E1B26300E1B26AE
:1023C00060003FF0D9FF600043F0DAFF60006FF07B
:1023D000DFFF0F06D8A010061150121013101410B2
:1023E000D8A4F5EF91F0F7EF91F0A4EF91F012007F
:1023F000800E07140D6EFF0E08140E6E010E0914E8
:102400000F6E000E0A14106E000ED2BE010E116E79
:102410000D5007180FE10E5008180CE10F50091865
:1024200009E110500A18D8B418EF92F01AEF92F0A0
:102430001DEF92F0FF0E64EF92F007C002F008C0AB
:1024400003F009C004F00AC005F0CAEC97F0600080
:1024500027F0F8FF600023F0F7FF60001FF0F6FFA1
:10246000000E126E12500B24D96E000E0C20DA6E84
:10247000DF50F56E7F0E1218D8A441EF92F043EFB3
:1024800092F046EF92F00C0047EF92F00D00122A06
:102490007F0E12644EEF92F050EF92F032EF92F016
:1024A0003901E5513F0B8009E56FE585D29E550E58
:1024B000E66FAA0EE66FE58311B002D0D29E01D07E
:1024C000D28E3901E595000E1200A1EF92F00EC0F8
:1024D00006F00FC007F010C008F011C009F010C0DE
:1024E00002F011C003F029EC98F002C00AF003C01A
:1024F0000BF0BDEC92F006500710D8A482EF92F0DA
:1025000084EF92F08AEF92F00EC00EF00FC00FF041
:10251000BCEF92F0010E0E24026E000E0F20036E2F
:10252000600043F0D9FF600047F0DAFFDF50126E21
:102530001250046E056A0CEC97F002C00EF003C056
:102540000FF00E500F10D8B4A8EF92F0AAEF92F04F
:10255000B8EF92F060003BF0D9FF60003FF0DAFF87
:10256000DF50D8A4B6EF92F0B8EF92F067EF92F098
:10257000000E0E6E000E0F6E1200FEEF92F0600065
:102580001BF0D9FF60001FF0DAFFDF50D8B4CBEFAB
:1025900092F0CDEF92F0E2EF92F0600023F0D9FFDD
:1025A000600027F0DAFF60001BF0E1FF60001FF021
:1025B000E2FFDE50E618D8B4E0EF92F0E2EF92F0DE
:1025C000FAEF92F060001BF0D9FF60001FF0DAFF15
:1025D000DF500C6E600023F0D9FF600027F0DAFFB7
:1025E000DF500D6E0D500C5C066E076AD8A0070612
:1025F0000FEF93F0064A072A084A092A0A06D8A0CC
:102600000B060A2806E10B28D8A409EF93F00BEF7C
:1026100093F0BFEF92F0000E076E000E066E1200F0
:10262000000E0A6E000E0B6E000E0C6E000E0D6E8C
:102630000650071008100910D8B421EF93F023EFCB
:1026400093F059EF93F0010E0E6E2DEF93F0D890AA
:1026500006360736083609360E2A09AE32EF93F0F1
:1026600034EF93F027EF93F0D8900A360B360C3600
:102670000D360650025C07500358085004580950A4
:102680000558D8A046EF93F048EF93F051EF93F040
:102690000650025E0750035A0850045A0950055A62
:1026A0000A80D89009320832073206320E2E34EFF3
:1026B00093F00AC002F00BC003F00CC004F00DC090
:1026C00005F01200800EF66E290EF76E010EF86E00
:1026D00000EE00F310EE80F009006F00D7FFEEFF70
:1026E000E550E150F9E1000EF66E290EF76E010E8D
:1026F000F86E00EE80F210EE80F009006F00D7FF58
:10270000EEFFE550E150F9E100EE80F316EE00F344
:10271000EE6AE550E150FCE1E250FAE100EE00F231
:10272000800EEE6AE806FDE100EE00F1D00EEE6AE2
:10273000E806FDE100EE60F05F0EEE6AE806FDE1FE
:1027400000EE45F0170EEE6AE806FDE1080ED56EC4
:10275000000ED66E000ED76E000100EF80F002C0B2
:1027600008F003C009F0D5EF93F00606D8A00706DD
:10277000600013F0D9FF600017F0DAFF044A052A61
:10278000600023F0E1FF600027F0E2FF084A092A19
:102790006F007FFFE7FFE750D8A4D1EF93F0D3EFAE
:1027A00093F0D5EF93F0EAEF93F006500710D8A41A
:1027B000DCEF93F0DEEF93F0B5EF93F0EAEF93F0F8
:1027C000600023F0D9FF600027F0DAFF000EDF6E13
:1027D000084A092A0606D8A00706062806E107289F
:1027E000D8A4F5EF93F0F7EF93F0E0EF93F0120039
:1027F0000650071008100910D8B401EF94F003EF49
:1028000094F033EF94F0010E0A6E0DEF94F0D8902F
:1028100006360736083609360A2A09AE12EF94F052
:1028200014EF94F007EF94F00650025C0750035841
:102830000850045809500558D8A021EF94F023EF10
:1028400094F02BEF94F00650025E0750035A0850A4
:10285000045A0950055AD890093208320732063214
:102860000A2E14EF94F002C002F003C003F004C07B
:1028700004F005C005F012003901A3A742EF94F05F
:1028800044EF94F047EF94F06F00A0F7BAF0BC8AE1
:10289000000E526E000E516E525009E17F0E515CD7
:1028A000D8A055EF94F057EF94F059EF94F065EFFE
:1028B00094F0000E5124D96E010E5220DA6E000EF3
:1028C000DF6E514A522A4CEF94F03901938D3D014D
:1028D000F289000EF96F000EFA6F000E0001BA6F58
:1028E000000E0101006F000E0001B56F000E526E68
:1028F000000E516E000EBA6FBC9A39019387120018
:10290000000102030405060708090A0B0C0D0E0F4F
:10291000101112131415161718191A1B1C1D1E1F3F
:10292000202122232425262728292A2B2C2D2E2F2F
:10293000303132333435363738393A3B3C3D3E3F1F
:10294000404142434445464748494A4B4C4D4E4F0F
:10295000505152535455565758595A5B5C5D5E5FFF
:10296000606162636465666768696A6B6C6D6E6FEF
:10297000707172737475767778797A7B7C7D7E7FDF
:1029800000100110021003100410051006100710AB
:10299000081009100A100B100C010D100E100F106A
:1029A000107F117F127F137F147F157F167F177F93
:1029B000187F197F1A7F1B7F1C7F1D7F1E7F1F7F43
:1029C00020802180228023802480258026802780EB
:1029D000288029802A802B802C802D802E802F809B
:1029E00030FF31FF32FF33FF34FF35FF36FF37FF53
:1029F00038FF39FF3AFF3BFF3CFF3DFF3EFF3FFF03
:102A0000000EBA6E430EC26E000E3A01406F000E09
:102A1000416F000E426F43694469BA96000EBB6E67
:102A2000C70EC36E000E506F000E096F000E5A6F76
:102A3000000E5B6F080EC06F030E516F000E526FD9
:102A400053695469000EBC6E890EC46E000E606F2F
:102A5000000E106F090E116F000E126F000E136F33
:102A6000000E146F000E156F130E166F170EE56F24
:102A7000BC8A000E626F0F0E636F64696169120099
:102A8000000E076E000E066E04500510D8B44BEF12
:102A900095F04DEF95F075EF95F0010E086E55EF3E
:102AA00095F0D89004360536082A05AE5AEF95F011
:102AB0005CEF95F051EF95F0D8900636073604504C
:102AC000025C05500358D8A068EF95F06AEF95F0C6
:102AD0006FEF95F00450025E0550035A0680D890BF
:102AE00005320432082E5CEF95F006C002F007C0F4
:102AF00003F01200600013F0F6FF600017F0F7FF1C
:102B0000000EF86E08006F00D4FFB0F0A1EF95F052
:102B1000600013F0F6FF600017F0F7FF000EF86E8C
:102B200008006F00D4FFB0F060000BF0D9FF600028
:102B30000FF0DAFF6000C3F2DFFF024A032A044A03
:102B4000052A0001B051D8A4A8EF95F0AAEF95F09E
:102B500088EF95F060000BF0D9FF60000FF0DAFF0E
:102B6000000EDF6E1200000E0001836F000E826FF8
:102B7000DCEF95F03901A3A9C0EF95F0C2EF95F015
:102B8000BAEF95F0000182512624D96E8351272097
:102B9000DA6EDF503D01EA6F0001824B832B8351D7
:102BA00009E1810E825DD8A0D8EF95F0DAEF95F0BB
:102BB000DCEF95F0EAEF95F082512624D96E83512F
:102BC0002720DA6EDF50D8A4E8EF95F0EAEF95F011
:102BD000BAEF95F012001CC024F01DC025F021BEF4
:102BE000F6EF95F0F4EF95F008EF96F0600073F0D3
:102BF000D9FF600077F0DAFF2D0EDF6E1C4A1D2A28
:102C0000211E201E1F1E1E6C000E1F2220222122AC
:102C10001CC00FF01DC010F01EC011F01FC012F03C
:102C200020C013F021C014F022C015F023C016F00C
:0E2C300069EC91F024C01CF025C01DF01200CC
:102C40003901A4A126EF96F028EF96F053EF96F005
:102C500094A12DEF96F02FEF96F053EF96F0000130
:102C600097BF3DEF96F0975106E19605D8B03BEF40
:102C700096F03DEF96F043EF96F0B29039019491C3
:102C8000598246EF96F09607D8A0970700018A4B25
:102C90008B2BCF0EB16E2C0EB06E000E956F010E09
:102CA000946F3901A49111000B500C10D8B45BEF54
:102CB00096F05DEF96F081EF96F0010E0D6E65EFE8
:102CC00096F0D8900B360C360D2A0CAE6AEF96F0C3
:102CD0006CEF96F061EF96F00B50095C0C500A58BF
:102CE000D8A075EF96F077EF96F07BEF96F00B504B
:102CF000095E0C500A5AD8900C320B320D2E6CEF34
:102D000096F009C009F00AC00AF012003901A7A123
:102D10008CEF96F08EEF96F0B3EF96F097A193EFCD
:102D200096F095EF96F0B3EF96F00001924B932B4F
:102D300091BFA3EF96F0915108E19005D8A0A3EFC1
:102D400096F0A5EF96F0AAEF96F09007D8A091071D
:102D5000ABEF96F05988000E8F6F010E8E6F390120
:102D6000A791FE0E9F6E110004C00AF005C00BF083
:102D700002C008F003C009F0D3EF96F060002BF01A
:102D8000D9FF60002FF0DAFFDF500C6E0A4A0B2AE1
:102D9000600023F0D9FF600027F0DAFF600033F015
:102DA000DFFF084A092A0606D8A00706062806E11A
:102DB0000728D8A4DEEF96F0E0EF96F0BEEF96F08D
:102DC0001200F9EF96F03901A3A9E9EF96F0EBEFC5
:102DD00096F0E3EF96F060000BF0F6FF60000FF066
:102DE000F7FF000EF86E08006F00D7FFEAFD024AF9
:102DF000032A60000BF0F6FF60000FF0F7FF000EF3
:102E0000F86E0800F5500009D8A409EF97F00BEF11
:102E100097F0E3EF96F0120060000BF0D9FF60002E
:102E20000FF0DAFF0450DE18D8A419EF97F01BEF6B
:102E300097F021EF97F002C002F003C003F035EFE6
:102E400097F060000BF0D9FF60000FF0DAFF024A44
:102E5000032ADF50D8A42FEF97F031EF97F00CEF53
:102E600097F0000E026E000E036E1200000E3D0180
:102E7000EC6F000EED6F000EEE6F000EEF6F000EA8
:102E8000F06F000EF16FB00EF26F800EF36F000E58
:102E9000F46F8A0EF56F000EF66F000EF76F000EDE
:102EA000F86F000EF96F000EFA6FF28BF289800E48
:102EB000F46F39019397120039019491050EB56EA4
:102EC000000EB26E000EB46EB28AB298B292B29494
:102ED000CF0EB16E2C0EB06ED29A84810001965145
:102EE0009711D8A476EF97F078EF97F07CEF97F0F2
:102EF000000E976F040E966F59923901A491B2900B
:102F00001200D28A000ED2BE010E026ED29E550E63
:102F1000D46EAA0ED46ED490000ED76E000ED66E6C
:102F2000080ED56E550ED46EAA0ED46ED48002B0A3
:102F30009CEF97F09FEF97F0D28EA0EF97F0D29E84
:102F40003901838781818481878112003901A1A1A0
:102F5000ACEF97F0AEEF97F0C6EF97F091A1B3EF1B
:102F600097F0B5EF97F0C6EF97F02A0E016E8E0E30
:102F7000E82EFED7012EFCD7CBA0C1EF97F0C3EF10
:102F800097F0C4EF97F0598E3901A19100018C4B55
:102F90008D2B1100000ED2BE010E066E600013F0E4
:102FA000F8FF60000FF0F7FF60000BF0F6FF39014B
:102FB000E5513F0B8009E56FE585E589D29E550E09
:102FC000E66FAA0EE66FE58306B002D0D29E01D06E
:102FD000D28E3901E595120006C002F007C003F059
:102FE00008C004F009C005F0BBEC98F00A6E010EB1
:102FF0000624026E000E0720036E000E0820046EE9
:10300000000E0920056EBBEC98F00B6E0A50066EA0
:103010000BC007F0120039019791050EA26E800EC9
:10302000A16E000E9E6E620EA06EFE0E9F6E5998EF
:10303000000E00018F6F000E8E6F39018781A791FE
:10304000000E0001936F000E926F39019781A08EE0
:10305000120002C004F003C005F031EF98F0044AFA
:10306000052A600013F0D9FF600017F0DAFFDF5087
:10307000D8A43DEF98F03FEF98F02FEF98F0025072
:10308000045C026E03500558036E12003F011E9946
:103090001E971E951E931E911E8F1E9B1F9F1F9D88
:1030A0002195219321813901A19D919DA19B919B06
:1030B0003F011D691C691B691F971F951F931F9175
:1030C0001200046E000E036E3A0E04606AEF98F070
:1030D0006CEF98F076EF98F02F0E046472EF98F092
:1030E00074EF98F076EF98F0010E036E03C002F0D3
:1030F000023012003901A3A980EF98F082EF98F016
:103100007AEF98F00D0E3D01EA6F3901A3A98BEF1C
:1031100098F08DEF98F085EF98F00A0E3D01EA6F78
:103120001200000EAC6EAC508F0B3009AC6EF00E7E
:10313000AC16B40EAB6E000EAA6E010EAE6E040E8F
:10314000AF6E39019495A495AC8E12000250040222
:103150006F00CCFF06F06F00D0FF07F002500502B1
:10316000F350072603500402F350072606C002F06E
:1031700007C003F012003901E5513F0B8009E56FEC
:10318000600013F0F8FF60000FF0F7FF60000BF035
:10319000F6FF0800F5501200599202C096F003C0E5
:1031A00097F0B282CF0EB16E2C0EB06E3901A491A1
:1031B0009481B2801200000E7E6E7E987E867E84A0
:1031C0007E927E903F015E935E81000E7F6E7E8ECA
:1031D0001200026E3901A3A9F0EF98F0F2EF98F017
:0C31E000EAEF98F060000BF0EAFD12002E
:020000040020DA
:10000000FF0FFF0FFF0FFF0FFF0FFF0FFF0FFF0F80
:020000040030CA
:0A0000008CFFEFF79FFFFFFFFFFFEB
:00000001FF
